S01F00002E2E5C62696E5C64656D6F70726F675F786D63343730302E73726563E9
S31508004000000002207D4F0008CB4F0008CD4F000866
S31508004010CF4F0008D14F0008D34F0008000000001A
S31508004020000000000000000000000000D54F000856
S31508004030D74F000800000000D94F00080D510008AE
S31508004040DF4F0008E14F0008E34F0008E54F00087E
S31508004050E74F0008E94F0008EB4F0008ED4F00084E
S31508004060EF4F0008000000000000000000000000FC
S31508004070F14F000800000000F34F0008F54F000854
S31508004080F74F0008F94F0008FB4F0008FD4F0008DE
S31508004090FF4F0008015000080350000805500008AB
S315080040A007500008095000080B5000080D5000087A
S315080040B00F5000081150000813500008155000084A
S315080040C017500008195000081B5000081D5000081A
S315080040D01F500008215000082350000825500008EA
S315080040E027500008295000082B5000082D500008BA
S315080040F02F5000083150000833500008355000088A
S3150800410037500008395000083B5000083D50000859
S315080041103F50000841500008435000084550000829
S3150800412047500008495000084B5000084D500008F9
S315080041304F500008515000085350000855500008C9
S3150800414057500008595000085B5000085D50000899
S315080041505F50000861500008635000086550000869
S315080041600000000000000000000000000000000041
S3150800417067500008695000086B5000086D50000829
S315080041806F500008715000087350000875500008F9
S3150800419077500008795000087B5000087D500008C9
S315080041A07F50000881500008835000088550000899
S315080041B087500008895000088B5000088D50000869
S315080041C08F50000891500008935000089550000839
S315080041D097500008995000089B50000800000000FE
S315080041E09D5000089F500008A1500008A3500008E1
S315080041F0A550000800000000A750000800000000B5
S31508004200EE11AA5510B5054C237833B9044B13B1F2
S315080042100448AFF300800123237010BD80000020FE
S3150800422000000000C4510008084B10B51BB108492E
S315080042300848AFF300800848036803B910BD074B68
S31508004240002BFBD0BDE81040184700BF0000000057
S3150800425084000020C4510008680000200000000007
S31508004260154B002B08BF134B9D46A3F5803A00213A
S315080042708B460F461348144A121A00F089FF0F4B53
S31508004280002B00D098470E4B002B00D098470020F3
S31508004290002104000D000D48002802D00C48AFF399
S315080042A0008000F04FFF2000290000F05DFE00F0BE
S315080042B035FF00BF000008000000022000000000D3
S315080042C000000000800000200C0100200000000013
S315080042D0000000002DE9F0438BB04FF461430193D1
S315080042E008238DF808308DF8093001258DF80A5015
S315080042F010278DF80B700026ADF80C601C4C01A930
S31508004300204600F007FD8DF81C6008954FF002095D
S315080043108DF82490DFF85C8007AA0421404600F057
S31508004320E5FA90238DF8103005958DF818900DEB69
S3150800433007020521404600F0D9FAE36923F007038E
S315080043402B43E3612B4604223946204600F06AFDDA
S315080043502B4604223146204600F07CFD236C23F0D0
S315080043600F0343EA090323640BB0BDE8F08300BFDB
S31508004370000003400081024830B58BB000F00CFB0A
S31508004380044600E06400414B9C42FBD900E0640807
S315080043903F4B9C42FBD8224601213E4800F0DAFBFF
S315080043A001943D4B02934FF4FA53ADF80C300123B8
S315080043B0ADF80E30394C01A9204600F005FB2368FC
S315080043C043F040032360236843F001032360344B22
S315080043D0344A1A60DA79022161F38712DA71596868
S315080043E040F2676060F31C0159609A6860F31C022A
S315080043F09A60090E6FF34511D971120E42F0200228
S31508004400DA7208221A73002305E0254A1A440021A5
S3150800441011740133DBB2072BF7D92148002505763D
S3150800442000F0F8FB012211461A4800F053FB1B4C1A
S31508004430236823F040032360236823F001032360E5
S315080044400AAA02F80C5D184D0D21284600F04EFA0E
S3150800445090238DF810300123059302238DF8183028
S3150800446004AA0C21284600F041FA236843F04003C9
S315080044702360E36823F0070343F00203E36023683D
S3150800448023F0400323600BB030BD00BFFF1AB7000E
S31508004490000E27070040014820A1070000430148F5
S315080044A0E00000202050014800810248074BD3F85D
S315080044B0143113F0080F07D110B50446034800F06D
S315080044C05FFC2070012010BD0020704700000340EB
S315080044D008B5FFF7FFFEFFF74FFF08BDBFF34F8F85
S315080044E00549CA6802F4E062044B1343CB60BFF384
S315080044F04F8F00BFFDE700BF00ED00E00400FA059E
S3150800450008B5174B1B785BB91648FFF7CFFF01288C
S3150800451024D10122124B1A700022134B1A7008BDBF
S31508004520114B1B7801330F481844FFF7BFFF0128CA
S3150800453014D10D4A13780133DBB21370094A127885
S3150800454093420BD10022064B1A70064B5B78FF2B61
S3150800455004D1044B9B780BB9FFF7C0FF08BD00BF19
S31508004560DE0000209C000020DD00002000B583B09E
S31508004570174B1B68DB6913F0010F1BD0144800F0BA
S3150800458093FB60B1002210E0114A1A44117C02AA7A
S315080045901A4402F8081C0133DBB2012201E00022AA
S315080045A013460B49097B8B42EED3094B1B68012145
S315080045B0D96100E0002242B19DF80030FF2B04D1FA
S315080045C09DF801300BB9FFF789FF03B05DF804FBCE
S315080045D0E000002008B5FFF793FFFFF7C7FF08BD07
S315080045E010B5054C80220821204600F07BFB4FF0D1
S315080045F08073636010BD00BF0085024808B500F0EF
S315080046007FFD0D4B1B68C31AB3F5FA7F13D30B4B0B
S315080046101B783BB90122094B1A704FF48072084B7C
S315080046205A6006E00022054B1A704FF08072044B60
S315080046305A60014B186008BD0001002004010020E3
S315080046400085024882B00023019303E000BF019B66
S3150800465001330193019B8342F8D302B0704700BF30
S3150800466072B60D4B0D4A9A60BFF34F8F62B6D3F8F8
S31508004670882042F47002C3F888205A6922F008029A
S315080046805A61074941F214028B5823F00F0343F08D
S3150800469004038B50704700BF00ED00E0004000089F
S315080046A00010005800487047001BB70010B51E4B95
S315080046B0DB6813F4803F27D01C4BDB6813F0010F2F
S315080046C002D1FFF7EFFF00E01948184B1B6813F0FB
S315080046D0040F11D015498A68C2F303628B68C3F3C5
S315080046E006238C68C4F30644611C02FB0112B0FB66
S315080046F0F2F203FB022208E00C4B9B6803F07F03EF
S315080047000133B0FBF3F200E0094A0749C868C0B2B2
S315080047100130B2FBF0F3086900F001000130B3FB89
S31508004720F0F0044B186010BD0046005010470050CA
S3150800473000366E016800002070B5574B1B6813F0F1
S31508004740010F09D1544A536843F001035360524B91
S315080047501B6813F0010FFAD0504B1B6813F4007F47
S3150800476008D04E4A936843F40073936041F64C5060
S31508004770FFF768FF4A4C636843F40023636040F61A
S31508004780C410FFF75FFF636823F4803323F0020346
S315080047906360444B5B6813F0300F21D0103C6368AC
S315080047A023F4702323F030036360FFF77BFF3E4B4F
S315080047B0A3FB00231B0D013B626842EA03436360C7
S315080047C0374BDA6822F00102DA605A6822F40032BE
S315080047D05A60334B1B6803F46073B3F5607FF8D1F6
S315080047E02F4B5A6842F001025A605A6842F010028A
S315080047F05A602E4A9A605A6842F040025A605A68CD
S3150800480022F010025A605A6842F480225A60244BF9
S315080048101B6813F0040FFAD0214A536823F00103EA
S3150800482053601F4B1B6813F0010FFAD1204C4FF051
S315080048300113E36000266661266126626662032329
S31508004840E3611C4BA3611C4BA362154D6B6823F0F7
S3150800485040036B60194BAB604FF41660FFF7F2FE2E
S31508004860174BAB604FF46160FFF7ECFE154BAB607E
S315080048704FF49650FFF7E6FE134BAB6041F27070AB
S31508004880FFF7E0FE114BAB604FF4E150FFF7DAFE9D
S315080048906660FFF70BFF70BD0042005000440050F1
S315080048A010470050004700506BCA5F6B002F0B0182
S315080048B0004600500500010003002001002F0501F5
S315080048C0002F0301002F0201002F0101002F000114
S315080048D010B54FF00053044C0FCB84E80F00FFF7D8
S315080048E0BFFEFFF729FF10BD6C000020F0B48B084F
S315080048F01F1D50F8276001F00305ED00F824AC40B1
S3150800490026EA040440F82740466F4F000324BC40BB
S3150800491026EA04044467194CA04203D004F58074BF
S31508004920A04207D1046E012606FA01F124EA010124
S31508004930016617E054688C404460CC08103450F87F
S31508004940247001F00701890007268E4027EA06062B
S3150800495040F8246050F82470167A06FA01F13943B3
S3150800496040F82410043350F82340117801FA05F270
S31508004970224340F82320F0BC704700BF008E02484F
S31508004980030F20F0704003EB43039A00014BD0500D
S31508004990704700BF14440050034B1868034B5B690B
S315080049A003F00103D8407047680000200046005015
S315080049B0030F20F0704003EB43039A00014BD050DD
S315080049C0704700BF484600502DE9F04142F2107E7C
S315080049D00027BC4601263BE00B6803EB83035A001D
S315080049E0B2FBF6F24D68B2FBF5F4394BA3FB048330
S315080049F0DB0803EB83034FEA4308C8EB0403052BE4
S31508004A0005D9334BA3FB0443DB08013303E0304BE2
S31508004A10A3FB0443DB0833B103EB83084FEA4804DE
S31508004A20B2FBF4F204E02A4BA3FB0232D2080123BC
S31508004A30AA4201D3521B00E0AA1A142B07D896459E
S31508004A4005D9B2F57A7F06D396461F46B44601368F
S31508004A50402EC1D901E01F46B44642F2107E012617
S31508004A60402212E042F2107302FB0333B3FBF7F362
S31508004A700C89A34201D31D1B00E0E51AAE4501D9F6
S31508004A80AE461646A34202D3013A022AEAD8BB1B0F
S31508004A90026842F040020260023B1B0303F4E04353
S31508004AA04A89013A9201D2B21343721E120202F4E3
S31508004AB0706213430CF1FF3C0CF03F0C43EA0C0305
S31508004AC00361036823F040030360BDE8F08100BF7B
S31508004AD0CDCCCCCCD0F8C43113F4407FFAD1013117
S31508004AE0120442F0020242EA0161C0F8C41170479A
S31508004AF038B50446074D2846FFF75AFF2846FFF7FC
S31508004B003FFF236823F001032360236813F0020F95
S31508004B10FBD138BD10000010D0F8C83123F00F03C0
S31508004B201943C0F8C8117047D0F8C80100F00F0043
S31508004B30704700BF08B5FFF7F7FF012802D0022823
S31508004B4003D005E0FFF728FF08BDFFF7ABFD08BD5A
S31508004B50002008BD70B504460E461546FFF7C8FF87
S31508004B6031462046FFF7D8FF2046FFF7E3FFB0FBA4
S31508004B70F5F1C1F58061002938BF002140F2FF3206
S31508004B80914228BF1146C1F58066B0FBF6F6AB091F
S31508004B9080099B02B3FBF0F3934228BF134603FB3D
S31508004BA000F0800AAA1BA5EB8010824200D80B46AB
S31508004BB0824201D8012100E00221E26822F4434240
S31508004BC022F0FF02E260E26843EA81331343E360BE
S31508004BD070BD00BF037E012B17D103682022DA615E
S31508004BE001680B6823F07062037B1B0603F0706391
S31508004BF013430B60036802691A61036842695A61C4
S31508004C000368034ADA61002070470320704700BF33
S31508004C1040002800016801F13842A2F5A83253097C
S31508004C20920A1B0203F4F85343EA42338A6822F4D1
S31508004C307F428A6001688A6813438B60037E012B72
S31508004C402FD810B503682022DA61C37913F0200F34
S31508004C500ED1426802F0604343EA824302689361D8
S31508004C60826802F0604343EA82430268D36005E043
S31508004C70036842689A6103688268DA600446037EBC
S31508004C80012B06D1FFF7A6FF23684FF00062DA6111
S31508004C9003E003684FF40062DA612368014ADA61C7
S31508004CA010BD70474000A0060368D969DA69C2F3E7
S31508004CB0800211F4006F0FD182B91A6902615A692C
S31508004CC04261D969DA69C2F3C00211F0040F07D04C
S31508004CD0002AF2D10020704703207047022070474F
S31508004CE00020704730B48B08043350F8235001F085
S31508004CF00301C900F8248C4025EA040440F823403F
S31508004D0050F823408A4044EA020140F8231030BC98
S31508004D10704700BF70B505460E4600F0E3F8F47913
S31508004D2004B9102422463168284600F035F8B379CC
S31508004D30013B64080134240244EA430343F4403344
S31508004D4043F00103EB633379013B1B0643F481739C
S31508004D506B6373792BB16A6B013B42EA03436B635E
S31508004D6005E06A6B3379013B42EA03436B634FF410
S31508004D70A063AB634FF0FF33EB6433892B6470BDDC
S31508004D80D0F80C3113F0E06F02D1406D80B2704755
S31508004D90D0F81C0180B2704763293BD9002A3BD062
S31508004DA02DE9F04115460C460646FFF7F5FD1B4969
S31508004DB0A1FB00377F09A1FB0431480940F2FF3EF9
S31508004DC04FF0010CE046714611E007FB01F300FBCA
S31508004DD005F2B3FBF2F39C0AC3F30903B4F5806F3B
S31508004DE004D29E4502D99E46A44688460139002922
S31508004DF0EBD148F4004333617269094B1340013D16
S31508004E0043EA85230CF1FF3C43EA0C437361002017
S31508004E10BDE8F08101207047012070471F85EB51DE
S31508004E20EF8000FC30B4D0F8084124F0E064C0F804
S31508004E300841D0F80851064C2C4041EA032343EABE
S31508004E40026244EA0203C0F8083130BC704700BF6A
S31508004E50C0C0FFF830B4D0F80C4124F0E064C0F8C4
S31508004E600C41D0F80C51074C2C4041EA032343EA85
S31508004E70026244EA020343F08053C0F80C3130BCA6
S31508004E80704700BFC0C0FFEF10B5114B984208D15C
S31508004E904FF40060FFF78CFD4FF40060FFF770FDDC
S31508004EA010BD0C4B984207D10B4C2046FFF780FDEE
S31508004EB02046FFF765FD10BD084B984206D1084C01
S31508004EC02046FFF775FD2046FFF75AFD10BD00BFC7
S31508004ED00800034008000248800000100840024805
S31508004EE00001001010B50446154B984203D003F58F
S31508004EF00073984203D11348FFF7C6FF14E0124B1C
S31508004F00984203D003F50073984203D10F48FFF780
S31508004F10BBFF09E00E4B984203D003F50073984295
S31508004F2002D10C48FFF7B0FF0323E360E36813F0F0
S31508004F30010FFBD0236C23F00F03236410BD00BFC1
S31508004F400000034008000340000002480800024829
S31508004F50004002480840024808B5FFF7A7FBFFF7DC
S31508004F603FFB00F0ABF808BD08B5FFF7F5FFFFF704
S31508004F70AFFAFFF743FBFFF72DFBFAE707498D4624
S31508004F800749084A084B9A42BEBF51F8040B42F833
S31508004F90040BF8E70548804705480047000002204B
S31508004FA0D05100080000002068000020D148000801
S31508004FB0614200083C493D4A002301E041F8043BB0
S31508004FC09142FBD3FFF7D0FFFEE7FEE7FEE7FEE7D9
S31508004FD0FEE7FEE7FEE7FEE7FEE7FEE7FEE7FEE79B
S31508004FE0FEE7FEE7FEE7FEE7FEE7FEE7FEE7FEE78B
S31508004FF0FEE7FEE7FEE7FEE7FEE7FEE7FEE7FEE77B
S31508005000FEE7FEE7FEE7FEE7FEE7FEE7FEE7FEE76A
S31508005010FEE7FEE7FEE7FEE7FEE7FEE7FEE7FEE75A
S31508005020FEE7FEE7FEE7FEE7FEE7FEE7FEE7FEE74A
S31508005030FEE7FEE7FEE7FEE7FEE7FEE7FEE7FEE73A
S31508005040FEE7FEE7FEE7FEE7FEE7FEE7FEE7FEE72A
S31508005050FEE7FEE7FEE7FEE7FEE7FEE7FEE7FEE71A
S31508005060FEE7FEE7FEE7FEE7FEE7FEE7FEE7FEE70A
S31508005070FEE7FEE7FEE7FEE7FEE7FEE7FEE7FEE7FA
S31508005080FEE7FEE7FEE7FEE7FEE7FEE7FEE7FEE7EA
S31508005090FEE7FEE7FEE7FEE7FEE7FEE7FEE7FEE7DA
S315080050A0FEE7FEE7FEE7FEE7800000200C01002091
S315080050B0014B1860704700BF0801002008B50C4B6B
S315080050C01B680C4AA2FB03239B09013BB3F1807FB3
S315080050D009D2094A5360FC21084B83F823100023A0
S315080050E09360072313600020FFF7E2FF08BD00BFA7
S315080050F068000020D34D621010E000E000ED00E0EB
S31508005100014B1868704700BF08010020024A13685F
S3150800511001331360704700BF0801002008B5074B2C
S31508005120044613B10021AFF30080054B1868836A63
S3150800513003B19847204600F033F800BF000000008E
S31508005140C051000870B50E4B0E4CE41AA410002589
S315080051501E46A54204D056F8253098470135F8E78B
S3150800516000F020F8084C094BE41AA41000251E4646
S31508005170A54204D056F8253098470135F8E770BDA2
S31508005180600000206000002064000020600000200D
S3150800519002440346934202D003F8011BFAE770471C
S315080051A0FEE70000F8B500BFF8BC08BC9E4670478D
S315080051B0F8B500BFF8BC08BC9E467047430000001F
S30D080051C00000002000000000B9
S30D080051C898F0FF7F01000000CA
S315080051D000000000000000000000000000000000C1
S315080051E000000000000000000000000000000000B1
S315080051F0BC5100080000000000000000000000008C
S315080052000000000000000000000000000000000090
S315080052100000000000000000000000000000000080
S315080052200000000000000000000000000000000070
S30D080052302942000805420008A6
S315080052380000000000000000000000000000000058
S309080052480000000054
S70508004000B2
